:0600000000008A01052842
:0800080009008330831681001A
:100010008B123930831290006030F8002B201028AA
:100020008312031306148316061083127A14C83041
:10003000F0000030F1003C208312031306108316F9
:10004000061083127A14C830F0000030F1003C2012
:1000500010286300292867308316031399001815A8
:1000600098168312181698170800F003700FF10AFB
:10007000F1037008710408000B110B1D3D28352099
:06008000031D3C280800EE
:00000001FF
